:020000040000FA
:020000000528D1
:0800080009008316FF2390009C
:1000100008308500003095000030810083120030E8
:100020008B0007309900363085000130A300A40012
:1000300003010C22C000F839031D26282022643059
:10004000A60085192A282A22A60B2128B9010F30DB
:100050001222A8210130A50025080C22B900403049
:100060002507840039088000A50A10302506031DE5
:100070002C280E30A60005140000051105122022C0
:1000800005162022A60B3E28051500000510A52008
:100090004019522841083106031D472842083206FC
:1000A000031D472845306F21031D58287A217528E4
:1000B0002318472849306F21031D6228A4188F2177
:1000C000851075284B306F21031D6A28A418472816
:1000D000051175284D306F21031D70289721752853
:1000E00047306F21031D47288F218C30A800A63090
:1000F000A90085198728B420AA002A188728400853
:10010000B00603198C280230300603199C28A90B6D
:100110007928A80B7728A1283508B7003608B80039
:100120000921AA002A18A12837083506031D9D2891
:1001300038083606031D9D2875288514000005150E
:10014000482885140000051547288519A528B420DE
:10015000AA002A18A52840083006031DA528092151
:10016000AA002A18A52800340A30A60052228519B0
:100170000134A60BB6285030A600851903290000CB
:100180000000000000000000A60BBD28C830A6003B
:100190008519F82800000000000000000000A60BF0
:1001A000C8280A30A6004C2285190134A60BD32892
:1001B000FA30A6008519E228000000000000A60B16
:1001C000DA2801340630A6004C22851D0134A60B26
:1001D000E4283A22851DF3283A22851D0134013096
:1001E000B000342200340330B0003A22342200340C
:1001F0000430A6004C22851D0134A60BFA280230DB
:10020000B0004C2200343A22851901340430B00089
:1002100000344019212930212A1801343908B1004D
:1002200030212A1801343908B20040182129302120
:100230002A1801343908B30030212A18013439084A
:10024000B40030212A1801343908B50030213908AA
:10025000B600401C00343506AA00AA0F0134003451
:10026000A601B9012A1440195229F930A000851DB0
:100270003F29000000000000A00B37290134C730DF
:10028000A00085194629A00B4129013440224018BD
:100290005222031085190314B90CA60AA61D35298C
:1002A000AA01003440220310851D0314B90CA60ACC
:1002B000A6196A29C730A00085196129A00B5C29FD
:1002C0000134C730A000851D6829A00B63290134C3
:1002D00052225229851D40224022AA010034840066
:1002E00000083506031D0134840A00083606031D84
:1002F00001340034A30B86290230A3000130A4008E
:100300000F300C22CF009D210514003405104F083A
:10031000B9000F3012220516000085160034A40B18
:1003200095290230A4000510003405140034CF0ACA
:100330000330CF054F060319CF014F18A12905122D
:10034000A2290516CF18A629851200348516003477
:10035000851DA8290530A600851220228516202299
:10036000A60BAC298519B229B420AA002A18B229F3
:10037000033030060319B2293008C0000921AA0051
:100380002A18B2290130A500303025078400000862
:10039000B90025081222A50A07302506031DC42925
:1003A0003108C1003208C20085120430A7003508A8
:1003B000B7003608B800A52040083006031DDB2929
:1003C0004019EA2941083106031DDB29420832069B
:1003D000031DDB2937083506031DF22938083606C8
:1003E0000319DB293508B90025081222A50A3608A9
:1003F000B90025081222A50A2708A6008516202282
:1004000085122022A60BFE29A70BD7294008B90088
:10041000030112228516003483169B001C141A084F
:100420008312080083169B0039089A001C1555306A
:100430009D00AA309D009C149C181C2A8312080061
:100440006430A200F930A0000000A00B242AA20B07
:10045000222A00340A30A100F930A0000000A00BCD
:100460002E2AA10B2C2A0034F930A0000000A00B8A
:10047000362A0034C730A0000000A00B3C2A00340C
:100480009530A0000000A00B422A00347C30A00070
:100490000000A00B482A00344A30A0000000A00B46
:1004A0004E2A00343130A0000000A00B542A003442
:0C04B0001830A0000000A00B5A2A0034F5
:02400E00C43FAD
:00000001FF
